:100000000C945D040C9485040C9485040C94850474
:100010000C9485040C9485040C9485040C9485043C
:100020000C9485040C9485040C94D2160C944117FE
:100030000C9485040C9485040C9485040C9485041C
:100040000C9485040C9485040C9485040C9485040C
:100050000C9485040C9485040C9485040C948816E7
:100060000C9485040C9485040C9485040C948504EC
:100070000C9485040C9485040C9485040C948504DC
:100080000C9473190C9485040C9485040C948504C9
:100090000C9485040C9485040C9485040C948504BC
:1000A0000C9485040C9485040C94850400000000D5
:1000B000003E5B4F5B3E3E6B4F6B3E1C3E7C3E1CEE
:1000C000183C7E3C181C577D571C1C5E7F5E1C0034
:1000D000183C1800FFE7C3E7FF0018241800FFE7EB
:1000E000DBE7FF30483A060E2629792926407F05AE
:1000F0000507407F05253F5A3CE73C5A7F3E1C1CC4
:1001000008081C1C3E7F14227F22145F5F005F5F83
:1001100006097F017F006689956A6060606060946F
:10012000A2FFA29408047E040810207E2010080874
:100130002A1C08081C2A08081E101010100C1E0C7F
:100140001E0C30383E3830060E3E0E060000000011
:100150000000005F00000007000700147F147F14F8
:10016000242A7F2A1223130864623649562050003D
:1001700008070300001C2241000041221C002A1C29
:100180007F1C2A08083E0808008070300008080814
:100190000808000060600020100804023E51494534
:1001A0003E00427F400072494949462141494D3352
:1001B0001814127F1027454545393C4A49493141B9
:1001C000211109073649494936464949291E000087
:1001D00014000000403400000008142241141414DC
:1001E0001414004122140802015909063E415D59C8
:1001F0004E7C1211127C7F494949363E41414122D1
:100200007F4141413E7F494949417F090909013EFA
:10021000414151737F0808087F00417F4100204021
:10022000413F017F081422417F404040407F021C33
:10023000027F7F0408107F3E4141413E7F0909094A
:10024000063E4151215E7F09192946264949493216
:1002500003017F01033F4040403F1F2040201F3FDC
:100260004038403F63140814630304780403615961
:10027000494D43007F4141410204081020004141A3
:10028000417F04020102044040404040000307084F
:100290000020545478407F2844443838444444284B
:1002A000384444287F385454541800087E090218F2
:1002B000A4A49C787F0804047800447D400020407A
:1002C000403D007F1028440000417F40007C0478BE
:1002D00004787C080404783844444438FC18242406
:1002E0001818242418FC7C08040408485454542486
:1002F00004043F44243C4040207C1C2040201C3C03
:100300004030403C44281028444C9090907C4464F9
:10031000544C44000836410000007700000041368C
:10032000080002010204023C2623263C1EA1A16112
:10033000123A4040207A3854545559215555794144
:100340002154547841215554784020545579400C1B
:100350001E527212395555555939545454593955FC
:100360005454580000457C410002457D420001453F
:100370007C40F0292429F0F0282528F07C545545AC
:10038000002054547C547C0A097F4932494949323F
:100390003248484832324A4848303A4141217A3A54
:1003A00042402078009DA0A07D39444444393D401E
:1003B00040403D3C24FF2424487E4943662B2FFCCB
:1003C0002F2BFF0929F620C0887E09032054547979
:1003D000410000447D413048484A32384040227A4A
:1003E000007A0A0A727D0D19317D2629292F2826C7
:1003F0002929292630484D402038080808080808CF
:100400000808382F10C8ACBA2F102834FA00007B27
:10041000000008142A142222142A1408950022002D
:1004200095AA005500AAAA55AA55AA000000FF00E7
:10043000101010FF00141414FF001010FF00FF1024
:1004400010F010F0141414FC001414F700FF000056
:10045000FF00FF1414F404FC141417101F10101FD5
:10046000101F1414141F00101010F0000000001FC3
:10047000101010101F10101010F010000000FF10CE
:100480001010101010101010FF10000000FF1400CA
:1004900000FF00FF00001F10170000FC04F41414FC
:1004A0001710171414F404F40000FF00F7141414C8
:1004B00014141414F700F7141414171410101F1048
:1004C0001F141414F4141010F010F000001F101F6B
:1004D0000000001F14000000FC140000F010F010D9
:1004E00010FF10FF141414FF141010101F00000050
:1004F00000F010FFFFFFFFFFF0F0F0F0F0FFFFFF54
:100500000000000000FFFF0F0F0F0F0F38444438AA
:10051000447C2A2A3E147E02020606027E027E02E5
:1005200063554941633844443C04407E201E200604
:10053000027E020299A5E7A5991C2A492A1C4C7241
:1005400001724C304A4D4D303048784830BC625AC8
:10055000463D3E494949007E0101017E2A2A2A2A58
:100560002A44445F444440514A444040444A514034
:100570000000FF0103E080FF000008086B6B0836F5
:1005800012362436060F090F060000181800000066
:100590001010003040FF0101001F01011E00191D55
:1005A0001712003C3C3C3C0000000000080B00021D
:1005B00002020000090400000102020000052400FC
:1005C000100105240101010424020605240600018E
:1005D0000705810310004009040100020A00000021
:1005E00007050202400000070583024000000403E3
:1005F000090412010002EF0201404123368000018C
:100600000102030141726475696E6F204C4C430016
:100610004142413133303600F0F89C8E8783878E1B
:100620009CF8F00000FEFF0303030303070EFCF831
:100630000000FEFF0303030303070EFCF80000FFA6
:10064000FF00000000000000FFFF0000FEFF8383AA
:10065000838383C7EE7C380000F8FC0E0703030396
:10066000070EFCF800003F7FE0C08080C0E07F3FC5
:10067000FFFF01010101010101FFFF0000FFFF0C6D
:100680000C0C0C1C3E77E3C100007FFFC0C0C0C053
:10069000C0E0703F1F00001F3F70E0C0C0C0E070AE
:1006A0003F1F00007FFFC1C1C1C1C1E3773E1C00F5
:1006B000001F3F70E0C0C0C0E0703F1F000000009E
:1006C0000001FFFF01000000D5F08D14A1C881CF0B
:1006D000D9F1AF2000484947482053434F524500C5
:1006E000040A0906000000000609090600000000CF
:1006F000020D09060000000060A090F0000000005C
:100700001826418182422418182444424222221C85
:100710003C4283818182621C265A81424181413E52
:100720000000C0300C0202020204040408F00000C1
:1007300000000003041820202020101008080700E3
:100740000080601008040202020202040830C000A7
:100750000001020C1020404040402010080403001B
:100760000000C0300C0404020204040C30C000007D
:10077000000F1020202020404040201008040300DB
:1007800000C0404040808060180402040830C0006F
:1007900000030C10202040404040242A1201010098
:1007A00003030201FFFEFDFEFF01020303FDFEFF46
:1007B0000102030201FFFEFD03030303030303FD24
:1007C000FDFDFDFDFDFDFDFDFDFD03030303030335
:1007D00000020303030404040303030200FEFDFDFF
:1007E000FDFCFCFCFDFDFDFEFCFCFDFDFDFE000234
:1007F0000303030404040303030200FEFDFDFDFCE8
:10080000FDFDFDFDFDFDFDFDFDFDFDFDFD03030306
:100810000303030303030303030201FFFEFDFD03C0
:100820000201FFFEFDFEFF010203FDFDFEFF0102CE
:1008300000EC05ED0AEF0EF211F613FB14001305A0
:10084000110A0E0E0A1105130014FB13F611F20E15
:10085000EF0AED05EC00EDFBEFF6F2F2F6EFFBED43
:1008600045524541534520444F4E4500574F524B4A
:10087000494E472E2E2E005354415254203D2052B3
:1008800049474854202B20420045524541534520BA
:100890004849474853434F52453F005041555345FF
:1008A000002000200018346E2E2E6E341841535450
:1008B00045524F4944530000ED1911241FBECFEF9C
:1008C000DAE0DEBFCDBF11E0A0E0B1E0E6EFFAE58F
:1008D00002C005900D92A434B107D9F728E0A4E432
:1008E000B1E001C01D92A135B207E1F714E0CDE5FA
:1008F000D4E004C02197FE010E94732DCC35D107AE
:10090000C9F70E941A1A0C94792D0C94000080915A
:10091000B1030895480F592F511D1416150684F57B
:10092000803891056CF597FF02C090E080E0413877
:10093000510514F040E850E0481BFB01E770FF2729
:1009400021E001C0220FEA95EAF777FF02C0695F54
:100950007F4FFB0133E0F595E7953A95E1F7F69582
:10096000FE2FEE27F795E795E80FF91FE351FC4FAF
:10097000415030F08191DF011197822B8C93F8CF99
:1009800008954F925F926F927F928F929F92AF9253
:10099000BF92CF92DF92EF92FF920F931F93CF936C
:1009A000DF9330E0F901E80FF91F1E161F060CF067
:1009B0007CC0803891050CF078C0602E712CF3015A
:1009C000E60FF71F1E161F060CF06FC0603471058E
:1009D0000CF06BC0E62FE7705E2EE7E06E0E711C28
:1009E000E3E075946794EA95E1F7F3E07595679510
:1009F000FA95E1F7062E000C770BDB01B695BA2FBE
:100A0000AA27B795A795A80FB91FA351BC4FEA0114
:100A1000F12CE12C6701C60ED71E48E0C416D104A4
:100A20000CF043C0EFEFCE16DE06A4F18C0150E0CF
:100A300040E04D01E0E88E0E911C17FD21C0FA0147
:100A4000EC0FFD1FA490B12C052C02C0AA0CBB1CFE
:100A50000A94E2F7EFEFCE16DE06C1F1FD01E40FD6
:100A6000F51F40804A284082552051F0E7E0CE161D
:100A7000D10431F0F401E40FF51FA080BA28B08250
:100A80004F5F5F4F0F5F1F4F421753071CF4003833
:100A9000110599F64FEFE41AF40AA058BF4FC20FA0
:100AA000D31F6E147F0409F0B5CFDF91CF911F9152
:100AB0000F91FF90EF90DF90CF90BF90AF909F90FD
:100AC0008F907F906F905F904F9008955110D2CF8C
:100AD000D7CFEDEEF3E0A0E0B8E000800EBC8111CE
:100AE000012C1197A0FDFDCF0192B9F70DB4089527
:100AF0002FB7F89483E08093E9009091E800892F64
:100B0000807295FF04C09091F20080E4891B2FBF92
:100B10000895FC018091EC03882311F13FB7F8940C
:100B200082E08093E9002091F200822F90E0181675
:100B3000190614F481E090E0882339F0289844E6FF
:100B40004093EB034091F1004083222339F0209140
:100B5000F200211103C02BE62093E8003FBF089567
:100B60008FEF9FEF08958091E30381110DC082E024
:100B70008093DF0384E08093E0031092E2031092FD
:100B8000E10381E08093E3038FED93E00895FC019E
:100B90000E94DB05319728F068517C4F8F4F9F4FA3
:100BA000F9CFAB01FC010E94DB05641775078E07C6
:100BB0009F07C8F30895ABEDB3E02FB7F8947D918C
:100BC0008D919C9166B52FBFA89B05C06F3F18F40F
:100BD0007F5F8F4F9F4F22E0660F771F881F991FFF
:100BE0002A95D1F70895AB01FC010E94DB05415025
:100BF0005109E109F10928F068517C4F8F4F9F4F4F
:100C0000F6CFAB01FC010E94DB05641775078E0768
:100C10009F07C8F3089540915C0150915D012091B8
:100C20005A0130915B0142175307B4F49091E800E8
:100C30009570E1F39091E80092FD19C08093F10066
:100C400080915C0190915D0101968F739927892BAA
:100C500019F48EEF8093E80080915C0190915D0122
:100C6000019690935D0180935C0181E0089580E09E
:100C70000895DF92EF92FF920F931F93CF93DF932C
:100C8000D82E8A01EB017B01E40EF51ECE15DF059F
:100C900059F0D7FE12C0FE0184910E940B062196E6
:100CA0008111F4CF0FEF1FEFC801DF91CF911F919A
:100CB0000F91FF90EF90DF9008958881EECF0F9312
:100CC0001F93CF93DF931F92CDB7DEB782E0898366
:100CD00042E450E06CEA75E080E80E9439060E9428
:100CE000B305DC0112960D911C910115110589F0D7
:100CF000D801ED91FC910280F381E02DBE016F5F80
:100D00007F4FC801099597FD04C0F8010085118542
:100D1000ECCF89810F90DF91CF911F910F910895B2
:100D2000615030F02091F100FC0120830196F8CF52
:100D3000289884E68093EB030895AF92BF92CF92F8
:100D4000DF92EF92FF920F931F93CF93DF936C018B
:100D50007B018B01040F151FEB015E01AE18BF086C
:100D6000C017D10759F06991D601ED91FC9101901E
:100D7000F081E02DC6010995892B79F7C501DF9136
:100D8000CF911F910F91FF90EF90DF90CF90BF9088
:100D9000AF9008958F929F92AF92BF92CF92DF92C1
:100DA000EF92FF920F931F93CF93DF936C017B0120
:100DB0008A0180910B01882309F45AC08091EC03C9
:100DC000882309F455C08091600180FF05C080919F
:100DD000E00082608093E000E801B12C8AEFA82E49
:100DE00093E0892E2AE3922E209711F4BB20C9F1BB
:100DF0000E947805811108C0AA94AA20C9F181E057
:100E000090E00E94C705F0CF8C171D0611F00CF082
:100E10008C2F9FB7F8948092E9002091E80025FD7F
:100E200002C09FBFE1CF282F30E0C21BD30BF701D8
:100E3000815020F041914093F100FACFE20EF31E71
:100E4000BB2021F09092E800B12CEBCF8091E8001C
:100E500085FDE7CF9092E800BB24B394209709F377
:100E6000F3CF5D9884E680935F01101611063CF085
:100E700081E090E0F6019383828310E000E0C801F6
:100E8000DF91CF911F910F91FF90EF90DF90CF9066
:100E9000BF90AF909F908F900895CF93DF931F9254
:100EA000CDB7DEB76983DC01ED91FC910280F3815F
:100EB000E02D41E050E0BE016F5F7F4F09950F903C
:100EC000DF91CF91089583E08093E9008091F20053
:100ED000882319F08AE38093E80008950E9478053A
:100EE00090E00895CF93DF931F92CDB7DEB7FC015A
:100EF0008485958597FD08C02FEF3FEF35872487C0
:100F00000F90DF91CF910895CE0101960E9489053F
:100F1000019719F4898190E0F3CF8FEF9FEFF0CF25
:100F20000F931F93CF93DF931F92CDB7DEB78C0142
:100F3000FC018485958597FF0BC0CE0101960E9428
:100F40008905019771F4898190E0F801958784877C
:100F5000F801848595850F90DF91CF911F910F91B6
:100F600008958FEF9FEFF1CFFC018485958597FD64
:100F70000BC09FB7F89482E08093E9008091F20063
:100F80009FBF90E0019608959FB7F89482E0809308
:100F9000E9008091F2009FBF90E0089520915301F5
:100FA000E0915101F0915201CF01029690935201CC
:100FB00080935101222319F08591949108958081A5
:100FC00091810895CF92DF92EF92FF92CF93DF93BA
:100FD0000E94CE07811520E8920791F4809171005C
:100FE0008D7F809371001092910046985F981092C7
:100FF0005001DF91CF91FF90EF90DF90CF90089557
:1010000021E020935001813020E8920751F4809133
:101010004E0190914F0190935201809351010E9493
:10102000CE0797FD05C020914D01222309F454C03D
:1010300020914C01211150C021E020935401EC017A
:10104000DF77209709F04BC081E0809355014698E7
:101050003FE9C32E3FE0D32EE12CF12CCAEFD0E0C4
:10106000E0914B08F0914C080995811103C081E093
:101070008093550180915401882329F08091550176
:10108000882309F43FC05F980E94CE070097F1F1D2
:101090009C01DE010E943C2DDC01CB0129E0B595CD
:1010A000A795979587952A95D1F7109290002AE0F9
:1010B00020939100D0929900C0929800809356019D
:1010C00090935701A0935801B093590180917100FA
:1010D0008260809371008DCF10925401B0CF9E0139
:1010E00050E040E060E472E48FE090E00E94E82C81
:1010F00069017A0181E0C81AD108E108F10810926B
:101100005501AECF4699BFCF5F9ABECF8FEF9FEF0D
:10111000DC01CBCF9C01E1E7F0E090819D7F9083E3
:1011200010925301EDE3F8E0F0935201E093510186
:10113000F0934F01E0934E013183208373836283E8
:1011400080E090E8958384830C94E20790E00C940F
:10115000C7058FB18095807F669B88601C9B8460EB
:1011600008951092B1033E98579808953E9A579A61
:1011700081E08093B103089590E1282F81E061FD23
:1011800084E060FD880F62FD8295687F969FD001A4
:101190001124A20FA351BC4F0C90082A40FF08262F
:1011A0000C9208958038910528F46034710510F48C
:1011B0000C94BC0808952F923F924F925F926F92C9
:1011C0007F928F929F92AF92BF92CF92DF92EF92D7
:1011D000FF920F931F93CF93DF93EC018B017A0162
:1011E0006901C61AD70AD7FE03C0D194C194D108A9
:1011F00047018C1A9D0A97FE03C09194819491082F
:101200008C149D0454F49E2D8F2D7901292F382F95
:101210009C2F8D2FE801092F182FEC16FD0654F492
:10122000902F812F8901292F382F9C2F8D2FE70197
:10123000E92EF82E17012C1A3D0A2901401A510AED
:1012400057FE03C0519441945108310137FE03C049
:101250008FEF681A780A759467948FEF0217130757
:101260000CF481E0A82E880FBB08EC16FD06A4F054
:1012700041E0BE01C8018C149D0414F0B801CE01F8
:101280000E94D2086418750877FE04C00A0D1B1D61
:10129000620C731C2196E9CFDF91CF911F910F91C2
:1012A000FF90EF90DF90CF90BF90AF909F908F9086
:1012B0007F906F905F904F903F902F9008952F9266
:1012C0003F924F925F926F927F928F929F92AF92D6
:1012D000BF92CF92DF92EF92FF920F931F93CF9323
:1012E000DF9300D000D000D01F92CDB7DEB76D30B5
:1012F000D9F030900D014090B4035090B503832D88
:1013000090E09F838E836A3051F51092B70310925C
:10131000B60323E0880F991F2A95E1F7480E591E5E
:101320005092B5034092B40381E090E027960FB647
:10133000F894DEBF0FBECDBFDF91CF911F910F910B
:10134000FF90EF90DF90CF90BF90AF909F908F90E5
:101350007F906F905F904F903F902F900895A09056
:10136000B603B090B70395E0699FB0011124FB016B
:10137000E455FF4F3F016501212CF5E02F1629F1BF
:10138000C3010196F301F491F9833C01420128E085
:101390002A83898181708D8310E000E00315D0F4E9
:1013A000F801EC0DFD1DFC83EB83F12CE12CE31423
:1013B00070F4B4016E0D7F1D4D818B819C810E9464
:1013C000D208FFEFEF1AFF0AF2CF1982DFCF0F5FCB
:1013D0001F4FE4CF2981269529838A8181508A83F2
:1013E000EE81FF818E0E9F1E8111D3CF2394CE0EEE
:1013F000DF1EF6E02F12C1CFC501329C800D911D7A
:1014000011249093B7038093B6038ECF682F8DE499
:1014100098E00C945F090F931F93CF93DF938C0197
:10142000D0E0C0E0F801EC0FFD1F6491662341F0AD
:101430008DE498E00E945F09892B11F02196F2CF8C
:10144000CE01DF91CF911F910F910895909162018C
:10145000982329F490916301982381E009F480E0B6
:101460000895CF93C82F0E94A908982F9C2381E04C
:101470009C1380E0CF9108952F923F925F926F92DC
:101480007F928F929F92AF92BF92CF92DF92EF9214
:10149000FF920F931F93CF93DF9300D000D000D023
:1014A000CDB7DEB77C018B01522E242F30E03E8376
:1014B0002D8381E090E05C01A21AB30AC9019195E5
:1014C000819591099C01220F331F3A8329836D81F5
:1014D0007E81600F711F452DC7010E94D208B8019F
:1014E0008D819E81681B790B452DC7010E94D20812
:1014F000452DB8018D819E818E0D9F1D0E94D208C1
:10150000452DB801C7012D813E81821B930B0E949E
:10151000D208D12CC12C81E090E09C838B83B7FC56
:101520000DC02D813E81215031093E832D8389815B
:101530009A8102969A838983A80EB91E9FEFC91AD1
:10154000D90A2B813C812E5F3F4F3C832B83A20E17
:10155000B31E36016E0C7F1C452D8D809E80800E43
:10156000911EB401C3010E94D20817012C183D0836
:10157000452DB401C1010E94D208452D48018D813D
:101580009E81881A990AB401C3010E94D208452D90
:10159000B401C1010E94D2084601800E911E452D62
:1015A000B4016D807E806E0C7F1CC3010E94D20846
:1015B000452DB40117012D813E81221A330AC10144
:1015C0000E94D20848018C189D08452DB401C30122
:1015D0000E94D208452DB401C1010E94D2088D811C
:1015E0009E81C816D9060CF49ACF26960FB6F894A9
:1015F000DEBF0FBECDBFDF91CF911F910F91FF9046
:10160000EF90DF90CF90BF90AF909F908F907F90A2
:101610006F905F903F902F90089580914A018823AA
:1016200021F010924A0180E008952091D703909113
:101630004B01322F391B932F30910C01931740F43B
:101640009F5F931790F491E093BF889513BE089520
:1016500081E080934A0120934B01E2EBF3E080812B
:10166000918101968083918381E008951092BB035C
:10167000E1ECF3E0178216821582148288E790E08D
:101680009093C0038093BF031092BE0310928E020A
:1016900010921F03109268030895EBECF3E080E0D2
:1016A00099E19183808388E893E1938382830E9408
:1016B000360B1092D4031092BD031092BC03089510
:1016C00080E19FEF9093C0038093BF0362E370E0DB
:1016D00086E990E00E948A088091CA038150809335
:1016E000CA03E1ECF3E080E099E19183808380E834
:1016F0009CE0938382831582148217821682089558
:10170000089590E080E008958F929F92AF92BF92EB
:101710000F931F93CF93DF93CDB7DEB7A1970FB68B
:10172000F894DEBF0FBECDBF19A2423008F44AE0E4
:101730008E010F5D1F4F842E912CB12CA12CA50181
:1017400094010E941A2DE62FB901CA01EA3044F52E
:10175000E05DD801EE938D01232B242B252B79F707
:1017600090E080E0109769F0FD0101900020E9F71A
:101770003197AF014A1B5B0BBD018DE498E00E94DD
:101780009D06A1960FB6F894DEBF0FBECDBFDF91C8
:10179000CF911F910F91BF90AF909F908F90089520
:1017A000E95CD7CFCF92DF92EF92FF92CF93DF9396
:1017B0006C01990FEE08FF08F7FE17C08DE20E943A
:1017C000060AEC0166277727CB016C197D098E0983
:1017D0009F094AE00E94840B8C0F9D1FDF91CF91DF
:1017E000FF90EF90DF90CF9008954AE0C701B601D7
:1017F000DF91CF91FF90EF90DF90CF900C94840B0E
:10180000FF920F931F93CF93DF93EC01F62E088185
:101810001981C8010E94C02CF81621F06F2DC80153
:101820000E94DA2CCE01DF91CF911F910F91FF9092
:1018300008950C94C02C0F931F93CF93DF938C01CA
:10184000EB010E94C02C8883C80101960E94C02C25
:101850008983CE01DF91CF911F910F910895CF928F
:10186000DF92EF92FF926B017C01C114D104E1047D
:10187000F10441F00E94682CA70196010E94E82C17
:101880006B017C01C701B601FF90EF90DF90CF9014
:101890000895AF92BF92CF92DF92EF92FF920F9393
:1018A0001F93CF93DF938091BF039091C00397FF65
:1018B00002C00C940F1600E019E0C02FD0E0A091F8
:1018C000C103B091C2036091C903062E000C770BCF
:1018D0009B012056384F80916803082E000C990B0D
:1018E000C817D9070CF09CC21C9FF0011D9FF00D7A
:1018F0001124E05EFC4F808191818A1B9B0BF901D2
:101900004491FC01E40FF11D47FDFA95E090C303FB
:10191000F090C403AB01485E5F4F1E161F060CF02B
:10192000D2C0F901D490FC01ED0DF11DD7FCFA9560
:10193000E43FF1400CF4D2C0F901D490FC01ED0D6C
:10194000F11DD7FCFA951E161F060CF0C1C1F90156
:101950002491DC01A20FB11D27FDBA951C9FF00157
:101960001D9FF00D1124E05EFC4F228133812E1962
:101970003F09FA01E056F84F44915901A40EB11CF9
:1019800047FDBA941A141B040CF0ADC1E491A901EF
:101990004E0F511DE7FD5A95A40FB51FAC3BB24049
:1019A0000CF4BDC0AB014053584FFA01F490FC0158
:1019B000EF0DF11DF7FCFA95DB01A85BBF4F1E167A
:1019C0001F060CF09AC1FA01D4905C01AD0CB11C59
:1019D000D7FCBA94E4EFAE16E1E0BE060CF49AC16F
:1019E000FA01D490FC01ED0DF11DD7FCFA951E16FD
:1019F0001F060CF0B5C1FA0144915C01A40EB11CA4
:101A000047FDBA94A501FD01E056F84FA491690184
:101A1000CA0ED11CA7FDDA94D6011A161B060CF0CB
:101A2000ABC1E4917901EE0EF11CE7FDFA94F701E8
:101A30004E0F5F1F4C3B52400CF471C0AB01405045
:101A4000584FFA01F490FC01EF0DF11DF7FCFA95E7
:101A500068587F4F1E161F060CF099C1FA01F490CA
:101A6000FC01EF0DF11DF7FCFA95E43FF1400CF499
:101A700099C1FA01F490FC01EF0DF11DF7FCFA9504
:101A80001E161F060CF0B5C1FA014491840F911D7A
:101A900047FD9A95FB01E056F84F44915901A40E79
:101AA000B11C47FDBA941A141B040CF0ACC1E491AC
:101AB0002E0F311DE7FD3A95820F931F8C3B92400C
:101AC00074F10F5FFACEF901D490FC01ED0DF11D18
:101AD000D7FCFA95ED30FE4F0CF42ECF1C9FF00191
:101AE0001D9FF00D1124E05EFC4FA281B381AE1961
:101AF000BF09FA01E056F84FD4905D01AD0CB11C5E
:101B0000D7FCBA941A141B040CF0D8C0E491AE0FA1
:101B1000B11DE7FDBA95A43FB1400CF00DCF62E3D3
:101B200070E086E990E00E948A080E94600B209194
:101B30001F032103F0011124E157FD4F1C9FC00139
:101B40001D9F900D1124EC01C05EDC4F88819981AE
:101B50002C813D81820F931F918380838A819B8199
:101B60002E813F81820F931F9383828364E670E00E
:101B700080E090E00E942F0C20911F032103F001D0
:101B80001124E157FD4F6253710981099109758351
:101B9000648364E670E080E090E00E942F0C209166
:101BA0001F032103F0011124E157FD4F6253710916
:101BB000810991097783668364E070E080E090E0BA
:101BC0000E942F0C20911F032103F0011124E157E3
:101BD000FD4F60872F5F20931F032103F001112425
:101BE000E157FD4F888199812C813D81820F931FA0
:101BF000918380838A819B812E813F81820F931FF5
:101C00009383828364E670E080E090E00E942F0C72
:101C100020911F032103F0011124E157FD4F62536E
:101C20007109810991097583648364E670E080E03D
:101C300090E00E942F0C20911F032103F00111243A
:101C4000E157FD4F625371098109910977836683DA
:101C500064E070E080E090E00E942F0C20911F0370
:101C60002103F0011124E157FD4F60872F5F20937E
:101C70001F03302F832F90E020916803422F022E04
:101C8000000C550B41505109841795070CF0C4C046
:101C9000189FD001199FB00D1124A05EBC4F019672
:101CA000189FF001199FF00D1124E05EFC4F812F69
:101CB00001900D928A95E1F73F5FDCCFE491AE0F82
:101CC000B11DE7FDBA95AD30BE4F0CF435CE27CF30
:101CD000F9012491DC01A20FB11D27FDBA95B19540
:101CE000A195B1093BCEE491A9014E0F511DE7FD2D
:101CF0005A955195419551094FCEFA01D4905C0106
:101D0000AD0CB11CD7FCBA94EDE0AE16EEEFBE06FA
:101D10000CF466CEFD01E056F84FF4905901AF0C7B
:101D2000B11CF7FCBA941A141B046CF4E491690119
:101D3000CE0ED11CE7FDDA94E4EFCE16E1E0DE062C
:101D40000CF04ECEECCEE4916901CE0ED11CE7FD35
:101D5000DA94FDE0CF16FEEFDF060CF441CEDFCEC5
:101D6000FA0144915C01A40EB11C47FDBA94A5018F
:101D700051954195510947CEE491D901AE0FB11D5E
:101D8000E7FDBA95FD01F195E195F10951CEFA0112
:101D9000F490FC01EF0DF11DF7FCFA95ED30FE4FCC
:101DA0000CF467CEFB01E056F84FA4915901AA0E3E
:101DB000B11CA7FDBA94D5011A161B066CF4E49168
:101DC0006901CE0ED11CE7FDDA94A4EFCA16A1E09A
:101DD000DA060CF04ECEA3CEE4915901AE0EB11C42
:101DE000E7FDBA94ADE0AA16AEEFBA060CF441CE08
:101DF00096CEFA014491840F911D47FD9A959195D5
:101E00008195910947CEE4912E0F311DE7FD3A955A
:101E100031952195310950CE21502093680351CE40
:101E200000E019E0C02FD0E02091C1033091C2033F
:101E30006091C903062E000C770BAB014056584F3A
:101E40006A0180911F03082E000C990BC817D9074F
:101E50000CF09BC21C9FF0011D9FF00D1124E15757
:101E6000FD4F80819181821B930BFA0124915C01CB
:101E7000A20EB11C27FDBA94E090C303F090C403F6
:101E8000DB0158961A141B040CF0D2C024915C019B
:101E9000A20EB11C27FDBA9440E9A41641E0B40695
:101EA0000CF4D2C0F60124915C01A20EB11C27FDF6
:101EB000BA941A141B040CF0C1C1C490AC014C0DAF
:101EC000511DC7FC5A951C9FF0011D9FF00D112458
:101ED000E157FD4F228133812E193F09FD01E05664
:101EE000F84FA4915901AA0EB11CA7FDBA94D501CF
:101EF0001A161B060CF0ACC1E4916901CE0ED11C80
:101F0000E7FDDA94F6014E0F5F1F483552400CF49E
:101F1000BCC0DB01A053B84FFD014491FC01E40FAC
:101F2000F11D47FDFA95AB01485B5F4F1E161F067A
:101F30000CF099C1FD01D4905C01AD0CB11CD7FC33
:101F4000BA94E0E9AE16E1E0BE060CF499C1FD01D9
:101F5000D490FC01ED0DF11DD7FCFA951E161F065D
:101F60000CF0B4C1FD01A4915C01AA0EB11CA7FD47
:101F7000BA94D501FA01E056F84F44916901C40EB4
:101F8000D11C47FDDA941C141D040CF0ABC1E49184
:101F9000A9014E0F511DE7FD5A95A40FB51FA83595
:101FA000B2400CF472C0AB014050584FFA01F490AB
:101FB000FC01EF0DF11DF7FCFA9568587F4F1E16D6
:101FC0001F060CF099C1FA01F490FC01EF0DF11D10
:101FD000F7FCFA95E039F1400CF499C1FA01F4905C
:101FE000FC01EF0DF11DF7FCFA951E161F060CF013
:101FF000B5C1FA014491840F911D47FD9A95FB01EB
:10200000E056F84F44915901A40EB11C47FDBA9413
:102010001A141B040CF0ACC1E4912E0F311DE7FD26
:102020003A95820F931F883592407CF10F5FFACE6C
:1020300024915C01A20EB11C27FDBA9441E7A416BD
:102040004EEFB4060CF42ECF1C9FF0011D9FF00D37
:102050001124E157FD4F228133812E193F09FD01E3
:10206000E056F84F44915901A40EB11C47FDBA94B3
:102070001A141B040CF0D8C0E4912E0F311DE7FD9B
:102080003A95203931400CF00DCF62E370E086E9DB
:1020900090E00E948A080E94600B20918E0221032A
:1020A000F0011124E259FE4F1C9FC0011D9F900DAD
:1020B0001124EC01C157DD4F888199812C813D812C
:1020C000820F931F918380838A819B812E813F8120
:1020D000820F931F9383828364E670E080E090E038
:1020E0000E942F0C20918E022103F0011124E2594D
:1020F000FE4F62537109810991097583648364E617
:1021000070E080E090E00E942F0C20918E0221036D
:10211000F0011124E259FE4F6253710981099109BE
:102120007783668364E070E080E090E00E942F0C8B
:1021300020918E022103F0011124E259FE4F6087A5
:102140002F5F20938E022103F0011124E259FE4FEC
:10215000888199812C813D81820F931F9183808397
:102160008A819B812E813F81820F931F938382837B
:1021700064E670E080E090E00E942F0C20918E02D7
:102180002103F0011124E259FE4F625371098109C4
:1021900091097583648364E670E080E090E00E94BA
:1021A0002F0C20918E022103F0011124E259FE4FE1
:1021B00062537109810991097783668364E070E055
:1021C00080E090E00E942F0C20918E022103F0010C
:1021D0001124E259FE4F60872F5F20938E02302F2B
:1021E000832F90E020911F03422F022E000C550BED
:1021F00041505109841795070CF0C3C0189FD001B6
:10220000199FB00D1124A157BD4F0196189FF001E1
:10221000199FF00D1124E157FD4F812F01900D9270
:102220008A95E1F73F5FDCCFE4912E0F311DE7FD8A
:102230003A9521373E4F0CF435CE27CFC490AC01F0
:102240004C0D511DC7FC5A955195419551093BCEF6
:10225000E4917901EE0EF11CE7FDFA94F701F19596
:10226000E195F10950CEFD01D4905C01AD0CB11C9B
:10227000D7FCBA94E1E7AE16EEEFBE060CF467CEDB
:10228000FA01E056F84FF4905901AF0CB11CF7FC7D
:10229000BA941A141B046CF4E4916901CE0ED11C9B
:1022A000E7FDDA94E0E9CE16E1E0DE060CF04FCE71
:1022B000ECCEE4916901CE0ED11CE7FDDA94F1E792
:1022C000CF16FEEFDF060CF442CEDFCEFD01A49167
:1022D0005C01AA0EB11CA7FDBA94D501B195A195D8
:1022E000B10948CEE491A9014E0F511DE7FD5A9561
:1022F00051954195510951CEFA01F490FC01EF0D31
:10230000F11DF7FCFA95E137FE4F0CF467CEFB01A7
:10231000E056F84FA4915901AA0EB11CA7FDBA943A
:10232000D5011A161B066CF4E4916901CE0ED11C7E
:10233000E7FDDA94A0E9CA16A1E0DA060CF04ECE69
:10234000A4CEE4915901AE0EB11CE7FDBA94A1E709
:10235000AA16AEEFBA060CF441CE97CEFA0144911C
:10236000840F911D47FD9A9591958195910947CECE
:10237000E4912E0F311DE7FD3A95319521953109F4
:1023800050CE215020931F0351CED0E0C9E06D2FD5
:1023900070E04091C1035091C2038091C903082E9F
:1023A000000C990BFC01E056F84F20918E02022E92
:1023B000000C330B621773070CF02BC1C69FD001C2
:1023C000C79FB00D1124A259BE4F2D913C91241BE3
:1023D000350B4491D901A40FB11D47FDBA951A16CA
:1023E0001B060CF039C0E491A9014E0F511DE7FD09
:1023F0005A95403951400CF439C0FC01E053F84F74
:102400004491D901A40FB11D47FDBA951A161B06B8
:102410000CF088C0E491A9014E0F511DE7FD5A95BB
:10242000403951400CF488C0FC01E050F84F449111
:10243000D901A40FB11D47FDBA951A161B060CF061
:10244000ABC0E4912E0F311DE7FD3A9520393140A4
:102450000CF4ABC0DF5F9BCFE491A9014E0F511D7F
:10246000E7FD5A9541375E4F0CF4C7CFC69FF00188
:10247000C79FF00D1124E259FE4F42815381E09134
:10248000C303F091C4034E1B5F0BFC01E854F84FEB
:10249000A4915A01AA0EB11CA7FDBA94D5011A162F
:1024A0001B06B4F5E4914E0F511DE7FD5A954039D6
:1024B00051400CF0A2CF68EC70E080E090E00E9408
:1024C000F3050E94600B3D2F832F90E020918E0238
:1024D000422F022E000C550B4150510984179507CD
:1024E0000CF093C0C89FD001C99FB00D1124A25910
:1024F000BE4F0196C89FF001C99FF00D1124E2590B
:10250000FE4F8C2F01900D928A95E1F73F5FDCCF53
:10251000E4914E0F511DE7FD5A9541375E4F0CF483
:102520006CCFC9CFE491A9014E0F511DE7FD5A951B
:1025300041375E4F0CF478CFC69FF001C79FF00D76
:102540001124E259FE4F42815381E091C303F0917F
:10255000C4034E1B5F0BFC01E851F84FA4915A01D4
:10256000AA0EB11CA7FDBA94D5011A161B0654F485
:10257000E4914E0F511DE7FD5A95403951400CF042
:1025800053CF99CFE4914E0F511DE7FD5A95413736
:102590005E4F0CF449CF8FCFE4912E0F311DE7FD34
:1025A0003A9521373E4F0CF455CFC69FF001C79F97
:1025B000F00D1124E259FE4F228133814091C30373
:1025C0005091C403241B350BFC01E85EF74F849146
:1025D0005901A80EB11C87FDBA94C5011816190639
:1025E00054F4E4912E0F311DE7FD3A952039314026
:1025F0000CF030CF60CFE4912E0F311DE7FD3A95FE
:1026000021373E4F0CF426CF56CF215020938E0217
:1026100021CF2091640130916501241B350B449139
:10262000B901640F711D47FD7A95AB016091C30339
:102630007091C403141615060CF04DC1E491A90164
:102640004E0F511DE7FD5A95403951400CF44DC1D4
:10265000FC01E053F84F44915901A40EB11C47FD11
:10266000BA941A141B040CF07FC1E491A9014E0F17
:10267000511DE7FD5A95403951400CF47FC1FC01D2
:10268000E050F84F44915901A40EB11C47FDBA9493
:102690001A141B040CF098C1E4912E0F311DE7FDB4
:1026A0003A95203931400CF498C18091CB03909138
:1026B000CC032091C1033091C203821B930B409144
:1026C000C903042E000C550BEA01C056D84FFE0179
:1026D0002491FC01E20FF11D27FDFA95A091C3039F
:1026E000B091C4032091CD033091CE03BA01685E4E
:1026F0007F4F1E161F060CF097C1FE01F490FC01DF
:10270000EF0DF11DF7FCFA95E43FF1400CF497C191
:10271000FE01F490FC01EF0DF11DF7FCFA951E1679
:102720001F060CF0DDC1FE01C4915C01AC0EB11CB2
:10273000C7FDBA94E5012A1B3B0BFB01E056F84F9D
:1027400064916901C60ED11C67FDDA941C141D0446
:102750000CF0D2C1E491B9016E0F711DE7FD7A95BD
:10276000C60FD71FCC3BD2400CF481C1BA016053D5
:10277000784FFB01C491FC01EC0FF11DC7FDFA95E8
:10278000DA01A85BBF4F1E161F060CF0BFC1FB018C
:102790001491FC01E10FF11D17FDFA95E43FF140A2
:1027A0000CF4BFC1FB011491FC01E10FF11D17FDF9
:1027B000FA951E161F060CF0DAC1FB016491EC01BC
:1027C000C60FD11D67FDDA95FD01E056F84F649103
:1027D0005901A60EB11C67FDBA941A141B040CF023
:1027E000D1C1E491B9016E0F711DE7FD7A956C0FAF
:1027F0007D1F6C3B72400CF43AC1BA016050784FB7
:10280000FB01C491FC01EC0FF11DC7FDFA9548587E
:102810005F4F1E161F060CF0BFC1FB01C491FC01E7
:10282000EC0FF11DC7FDFA95E43FF1400CF4BFC178
:10283000FB01C491FC01EC0FF11DC7FDFA951E16BA
:102840001F060CF0D9C1FB016491860F911D67FD35
:102850009A95FA01E056F84F44915901A40EB11C23
:1028600047FDBA941A141B040CF0D0C1E4912E0F4A
:10287000311DE7FD3A95820F931F8C3B92400CF47B
:10288000F6C08091680381111BC080911F038111E4
:1028900017C080918E02811113C08091BF03909167
:1028A000C00397FD0DC020916D01211109C0019752
:1028B000181619060CF0BDC19093C0038093BF0396
:1028C000DF91CF911F910F91FF90EF90DF90CF900C
:1028D000BF90AF900895E491A9014E0F511DE7FDFF
:1028E0005A9541375E4F0CF4B3CE4091660150913A
:1028F0006701461B570BFC01E854F84FA491EA010D
:10290000CA0FD11DA7FDDA951C161D0624F5E4910A
:102910004E0F511DE7FD5A95403951400CF098CEAD
:1029200068EC70E080E090E00E94F3050E94600B8C
:1029300010926C0110926B0110926A011092690161
:102940001092680110926701109266011092650161
:1029500010926401AACEE4914E0F511DE7FD5A95E5
:1029600041375E4FECF674CEE491A9014E0F511D34
:10297000E7FD5A9541375E4F0CF481CE40916601D8
:1029800050916701461B570BFC01E851F84FA49189
:10299000EA01CA0FD11DA7FDDA951C161D0654F4D5
:1029A000E4914E0F511DE7FD5A95403951400CF40A
:1029B000B7CF65CEE4914E0F511DE7FD5A954137D3
:1029C0005E4F0CF0ADCF5BCEE4912E0F311DE7FDD5
:1029D0003A9521373E4F0CF468CE20916601309134
:1029E0006701261B370BFC01E85EF74F8491A901B4
:1029F000480F511D87FD5A95CA011816190654F43F
:102A0000E4912E0F311DE7FD3A95203931400CF449
:102A100087CF4BCEE4912E0F311DE7FD3A9521373C
:102A20003E4F0CF442CE7CCFFE01F490FC01EF0D42
:102A3000F11DF7FCFA95ED30FE4F0CF469CE8901DB
:102A40000A1B1B0BFB01E056F84FF4905801AF0C2A
:102A5000B11CF7FCBA941A141B04CCF5E4910E0FC8
:102A6000111DE7FD1A95043F11400CF051CE68ECA2
:102A700070E080E090E00E94F3050E94600B1092ED
:102A80006C0110926B0110926A0110926901109210
:102A90006801109267011092660110926501109210
:102AA00064011092D3031092D2031092D1031092BA
:102AB000D0031092CF031092CE031092CD03109248
:102AC000CC031092CB038FEF80936D01DACEE491AB
:102AD0000E0F111DE7FD1A950D301E4F44F618CE4E
:102AE000FE01C4915C01AC0EB11CC7FDBA94E501B6
:102AF000D195C195D1091FCEE491B9016E0F711D19
:102B0000E7FD7A957195619571092ACEFB011491C3
:102B1000FC01E10FF11D17FDFA95ED30FE4F0CF4AD
:102B200041CEFD01E056F84FC4915901AC0EB11CE5
:102B3000C7FDBA94E5011C161D066CF4E491690109
:102B4000CE0ED11CE7FDDA9404EFC01601E0D006EA
:102B50000CF48DCF27CEE491E901CE0FD11DE7FD16
:102B6000DA95FE01ED30FE4F0CF081CF1BCEFB015C
:102B70006491EC01C60FD11D67FDDA95D195C19521
:102B8000D10922CEE491B9016E0F711DE7FD7A954E
:102B90007195619571092BCEFB01C491FC01EC0F7D
:102BA000F11DC7FDFA95ED30FE4F0CF441CEFA0150
:102BB000E056F84FA491E901CA0FD11DA7FDDA959F
:102BC0001C161D066CF4E4915901AE0EB11CE7FD14
:102BD000BA9404EFA01601E0B0060CF448CF28CE5A
:102BE000E491D901AE0FB11DE7FDBA95FD01ED30BD
:102BF000FE4F0CF03CCF1CCEFB016491860F911D63
:102C000067FD9A9591958195910923CEE4912E0FB8
:102C1000311DE7FD3A953195219531092CCE01966C
:102C200029F09093C0038093BF032BCE88E790E0F8
:102C3000F8CF88E790E09093C0038093BF03809122
:102C4000BB0388301CF48F5F8093BB03C0E019E0A6
:102C50008091BB03C8170CF033CE68EE7CE180E0B6
:102C600090E00E942F0C209168032103F0011124B1
:102C7000E05EFC4F60587A4D7183608368E670E1D6
:102C800080E090E00E942F0C209168032103F00166
:102C90001124E05EFC4F60547D4E7383628364E6D2
:102CA00070E080E090E00E942F0C209168032103E7
:102CB000F0011124E05EFC4F625371098109910912
:102CC0007583648364E670E080E090E00E942F0CDE
:102CD000209168032103F0011124E05EFC4F625350
:102CE0007109810991097783668364E070E080E06F
:102CF00090E00E942F0C209168032103F001112421
:102D0000E05EFC4F60872F5F20936803CF5FA0CF0A
:102D10000F920FB68F939F93EF93FF938091D603FB
:102D20008D5F8D3708F08D578093D603E7EDF3E084
:102D300080818E4F808391819F4F918382818F4FBD
:102D4000828383818F4F8383EBEDF3E080818F5FFC
:102D5000808381818F4F818382818F4F82838381A2
:102D60008F4F83838FB18F6066991C9B88278F3626
:102D700081F48091D503981B963068F0E0E0F8E08C
:102D800087E78083818388E180936000F09360000F
:102D9000FFCF9093D503FF91EF919F918F910FBE3D
:102DA0000F9018951F920F920FB60F9211248F93C8
:102DB0009F938091E1009091E100937F9093E100D7
:102DC00083FF0FC01092E90091E09093EB00109206
:102DD000EC0092E39093ED001092EC0398E0909356
:102DE000F00082FF22C093E09093E9009091F200FE
:102DF000992319F09AE39093E80090915F01992349
:102E000041F090915F01915090935F01911101C049
:102E10005D9A9091EB03992341F09091EB039150CF
:102E20009093EB03911101C0289A84FF18C0809100
:102E3000E2008E7E81608093E2008091E1008F7ECF
:102E40008093E100809160018E7E806180936001BB
:102E50009F918F910F900FBE0F901F90189580FF3C
:102E6000F7CF8091E2008E7E80618093E2008091B6
:102E7000E1008E7E8093E100809160018E7E816012
:102E8000E5CF1F920F920FB60F921124CF92DF92CF
:102E9000EF92FF920F931F932F933F934F935F9364
:102EA0006F937F938F939F93AF93BF93EF93FF9312
:102EB000CF93DF93CDB7DEB76C97DEBFCDBF109257
:102EC000E9008091E80083FF25C068E0CE014596C7
:102ED0000E94900682EF8093E8008D8987FF39C0B9
:102EE0009091E80090FFFCCF982F907609F034C1C4
:102EF0009E894F89588D2F89F88C911131C0803867
:102F000061F5809161018093F1001092F1008EEFE4
:102F10008093E8006C960FB6F894DEBF0FBECDBF6D
:102F2000DF91CF91FF91EF91BF91AF919F918F91E1
:102F30007F916F915F914F913F912F911F910F91D1
:102F4000FF90EF90DF90CF900F900FBE0F901F90EB
:102F500018959EEF9093E800C7CF1092F100D5CF5F
:102F6000913059F48111D3CF4130510581F68091D0
:102F700061018D7F80936101CACF933049F4811143
:102F8000C6CF4130510519F6809161018260F2CFC0
:102F9000953041F48091E80080FFFCCF20682093B9
:102FA000E300B5CF963009F0A9C00B8D1C8D22E04F
:102FB0001092E90010925D0110925C01F2122EC095
:102FC00010925B0110925A010E945F061F8299E0E5
:102FD0009983FA8291E09E8390EA98879AEF998785
:102FE00020915C0130915D01275F3F4F3C832B8333
:102FF0008D831092E90010925D0110925C01109394
:103000005B0100935A0149E050E0BE016F5F7F4FC2
:1030100080E00E9439060E945F0679CF10935B0121
:1030200000935A010E94B305DC0112960D911C9188
:103030000115110509F451C1D801ED91FC910480ED
:10304000F581E02DBE016B5E7F4FC80109950097A9
:1030500009F03EC1F80100851185EACFF3E0FF12C7
:103060000EC08F89882309F440C0823061F440E8A3
:1030700067E080E196E00E94BA19811148CF81E2B1
:103080008093EB0047CF813029F440E86BE084E087
:1030900096E0F1CF833099F70E94B305DC011296D8
:1030A000ED90FC908E010F5F1F4F6801E114F10459
:1030B00079F0D701ED91FC910680F781E02DB80100
:1030C000C7010995080F111DF701E084F184EECFC7
:1030D000D8011C92F60101900020E9F73197BF0159
:1030E0006C197D0940E0C601C6CF6EEE75E0FB01AC
:1030F000449150E080E80E94390609CF973009F4E6
:10310000BECF983021F481E08093F10000CF993058
:1031100009F0FDCE837009F0B2CFE3E1F1E081E088
:1031200031E096E32191222371F08093E9003093FE
:10313000EB00DF0111972C912093EC009093ED00B0
:103140008F5F873079F78EE78093EA001092EA006C
:103150008F898093EC03DBCE8B8D9C8D1092E900E0
:1031600010925D0110925C0190935B0180935A0173
:10317000898D811192C08E899D89913A49F481325D
:1031800009F07DCF47E050E064E071E080E0B3CF2C
:10319000913209F074CF833269F48F89988DB0E051
:1031A000A0E08093000190930101A0930201B093ED
:1031B0000301ADCE803269F48091E80082FFFCCF3C
:1031C00067E084E091E00E9490068BEF8093E80036
:1031D0009ECE823209F09BCE8F8980930B01EEEF59
:1031E000FFE7859194918B3F9C4D51F1E0E0F8E031
:1031F0008091040190910501A0910601B091070111
:10320000803B9440A105B105F1F480910B0180FD54
:103210001AC0EE3F8AE0F80789F587E797E79183C0
:1032200080838091600080935E0188E19BE00FB60F
:10323000F894A895809360000FBE9093600067CECD
:10324000EEEFFAE0D5CF808191818737974709F07B
:103250005ECEA89580916000886180936000809127
:103260005E0180936000EE3F2AE0F20789F08091D2
:10327000FE0A9091FF0A9183808349CE80819181DB
:103280008737980751F29093FF0A8093FE0AC5CFC3
:103290001092FF0A1092FE0A3ACE0E94B305DC019A
:1032A00012960D911C910115110509F4E8CED80173
:1032B000ED91FC910190F081E02DBE016B5E7F4F9E
:1032C000C8010995811123CEF80100851185EBCF46
:1032D000181619060CF41BCED2CEF1E0FF12BECEAA
:1032E00062EF75E004CF1F920F920FB60F92112478
:1032F0002F933F934F935F936F937F938F939F93FE
:10330000AF93BF93EF93FF93809156019091570134
:10331000A0915801B09159010097A105B10539F16B
:1033200020915501211105C0369A20915401211197
:103330004F9A0197A109B109B7FD08C080935601C2
:1033400090935701A0935801B0935901FF91EF91C9
:10335000BF91AF919F918F917F916F915F914F91AD
:103360003F912F910F900FBE0F901F9018950E94C4
:10337000E207ECCFEF92FF920F931F93CF93DF936F
:10338000F82E192FE62E042F81E0860F880F0E9459
:103390000B0683E00E940B06CF2DD12FEC0EFD2EE5
:1033A000F11CCE15DF05B9F007FF13C0FE018491B3
:1033B0000E940B06182F80E00E940B0681232196A5
:1033C0008111EFCFDF91CF911F910F91FF90EF907F
:1033D00008958881EDCF81E0F5CFEDEEF7E013821F
:1033E000128288EE93E0A0E0B0E084839583A68308
:1033F000B7838DE191E0918380838FEF9FEF958775
:103400008487EDE4F8E0138212828FE291E09183E9
:10341000808387E894E090934C0880934B0880E089
:1034200090E890934A088093490846983E9A5F989E
:10343000579A0895CDB7DEB76C97DEBFCDBF7894AD
:1034400083E084BD83E085BD81E080936E00E1E888
:10345000F0E083E08083E0E881E08083E1E983E0DD
:103460008083E0E981E08083E1EC87E08083E3EC26
:1034700081E08083E0EC82E08083E2EC81E0808385
:10348000EAE787E08083806880831092EC031092E3
:103490006101109260018091D70081608093D70014
:1034A00080EA8093D80089B5806189BD89B5826042
:1034B00089BD09B400FEFDCF81E090E00E94C70500
:1034C0008091D8008F7C80618093D8008091E0004B
:1034D000807F8093E0008091E1008E7E8093E10008
:1034E0008DE08093E200559A209A81EC80937C00D5
:1034F00081E785B987E684B985E38BB98FE38AB91B
:10350000769A6E9880EF81BB10BA80E58CBD81E021
:103510008DBD85E00E94A608599A85E00E94A60804
:103520005C98E8ECF6E085918EBD00000DB407FED6
:10353000FDCFE53DC1F75C9A81E88093640081E0AE
:103540008093650080E00E94690580E80E94310A4E
:103550008823A9F05C9885EA8EBD00000DB407FEB3
:10356000FDCF5C9A2E9858982D98809164008062C7
:103570008093640081E083BF889513BEFCCF84E014
:103580000E94310A8823B9F12D9884E80E94310AFB
:103590008823A1F02D9A88EC0E94A60858986FEF16
:1035A00082E090E00E94C82C84EF91E00E94C70561
:1035B000589A84E80E94310A8111FBCF84E10E946D
:1035C000310A8823A1F02D9A88EC0E94A6082E9833
:1035D00060E082E090E00E94C82C84EF91E00E94BD
:1035E000C7052E9A84E10E94310A8111FBCF88EC35
:1035F0000E94A608C4CF2D9A82E090E00E94190C88
:10360000882309F4D9C00E94B60881E090E00E94A6
:10361000C02C182F147081FF0EC011112E98F1EFDD
:10362000EF2EFF24FA9480E40E94310A882309F4E3
:10363000C6C02E9A589A82E30E94A6080E94A90842
:103640008111F9CF809164008E7F80936400809116
:103650007A00806480937A0080917A0086FDFCCFA6
:1036600000917800109179000E94DB05AB01BC014C
:10367000C801B0E0A0E0DC01992788278C019D01FA
:10368000040F151F261F371FC901B80120916400C0
:10369000216020936400611571058105910511F089
:1036A0000E94B72C81E280930C010E944D0B809107
:1036B000B103882309F4E0C00E94B60881E00E94AB
:1036C00069058FEF9FEF9093FA078093F9071091A8
:1036D000D40381E2113019F082E3111182E4809366
:1036E0000C010E940D0B882309F45EC0123011F406
:1036F0000C946C2908F0C3C0112309F43AC11130AD
:1037000009F40BC28091B1038823D9F142E06EE342
:1037100070E08DE790E00E948A0442E06FE370E081
:103720008DE790E00E948A0441E06EE370E08DE74F
:1037300090E00E94D20841E06FE370E08DE790E0F6
:103740000E94D20841E06EE370E08EE790E00E94B4
:10375000D20841E06FE370E08EE790E00E94D2086B
:103760002FE330E04EE750E06BE370E08EE790E04F
:103770000E94DB0841E06CE370E08FE790E00E947C
:10378000BC0840E054E06DEE73E08DEE97E00E94DF
:10379000CA0681E00E9469058091630180936201FD
:1037A0000E94A9088093630180E090E0892B09F4CE
:1037B0008ECF0E9400008BCF0E94B10826CF11232C
:1037C00031F004E0E016F10411F42E9A589881E0EB
:1037D0000E94690500E128E548E156E0B70184E16F
:1037E00090E00E94C10480E00E9469058FE00E9481
:1037F000A6082FEFE21AF20A39E1E316F10409F004
:1038000012CF112311F0589A2D9880E991E00E946F
:10381000C7052D9A81E090E00E94C02C80FF0BCF5D
:103820008AE090E00E94C02C9FEF980F9E3F08F026
:1038300002CF22E330E03093B7032093B60328E3AE
:1038400030E03093B5032093B4030AE010E0682F12
:103850008DE498E00E945F090F5F1F4FC8010E942E
:10386000C02C0031110599F780E00E94690588EEAF
:1038700093E00E94C705DFCE0E94B1081FCF14302D
:1038800011F40C94B12B10F40C94282B153009F082
:1038900039CF0EE010E01093B7030093B60380E237
:1038A00090E09093B5038093B40381E080930D0181
:1038B00089E898E00E940B0A1093B7030093B603BF
:1038C00088E290E09093B5038093B40387E798E093
:1038D0000E940B0A84E40E94310A882309F440C044
:1038E00004E610E084E2C82ED12C90E2E92EF12CFF
:1038F000D092B703C092B603F092B503E092B4033E
:103900008CE698E00E940B0A81E00E9469051A8308
:1039100009836FEFCE0101960E94000C0F5F1F4FCD
:103920000738110529F764EF71E080E090E00E940C
:10393000F305F092B703E092B603F092B503E0927C
:10394000B40380E698E00E940B0A81E00E946905BA
:1039500068EE73E080E090E00E94F3051092D403DB
:1039600088E00E94260A882309F4CCCE1092D40362
:10397000C9CE8AE090E09093B7038093B60390930A
:10398000B5038093B40382E080930D018DEA98E043
:103990000E940B0A8091CB039091CC032091CF031E
:1039A0003091D003820F931F9093CC038093CB036D
:1039B0004091CD035091CE032091D1033091D20399
:1039C000240F351F3093CE032093CD03893C12E39F
:1039D000910734F0885E95439093CC038093CB039A
:1039E0008091CB039091CC038C304EEF940734F44C
:1039F00088519A4C9093CC038093CB03253F5AE196
:103A0000350734F0285E3C413093CE032093CD033C
:103A10008091CD039091CE038C306EEF960734F4F5
:103A20008851934E9093CE038093CD038091B2033F
:103A30009091B3036EE170E00E944B2D892BE1F46D
:103A400064E670E080E090E00E942F0C6253710900
:103A5000810991097093D0036093CF0364E670E00D
:103A600080E090E00E942F0C625371098109910956
:103A70007093D2036093D1038091CD039091CE03D4
:103A800024E630E0B9010E945F2DFB01349780915C
:103A9000CB039091CC03B9010E945F2DCB0108E0CC
:103AA00028E045EA58E0BF0104970E94C10484E081
:103AB0000E94260A8823A1F083E08093CA0380E055
:103AC00099E19093C2038093C10380E89CE09093B6
:103AD000C4038093C3030E94360B81E08093D40318
:103AE00080E80E94260A811105C080E10E94260A12
:103AF000882331F08091B103882361F00E94B108DE
:103B000088E00E94260A882309F4FCCD83E0809394
:103B1000D403F8CD0E94B608F3CF8091CA031816DB
:103B200014F00C9461298091BF039091C0038938EF
:103B30009F4F0CF456C48091B20380FD4CC080E2CC
:103B40000E94310A882329F08091C9038150809313
:103B5000C90380E40E94310A882329F08091C903B7
:103B60008F5F8093C9038091C90388311CF088510D
:103B70008093C9038091C90387FF03C0885E809347
:103B8000C90380E80E94310A882329F1E091C90322
:103B90008E2F880F990BFC01E05DF74FE491209187
:103BA000C5033091C6032E0F311DE7FD3A953093C2
:103BB000C6032093C503FC01EF5CF74FE4918091AD
:103BC000C7039091C8038E0F911DE7FD9A959093BE
:103BD000C8038093C70380E10E94260A8823D1F09E
:103BE0006CE271E080E090E00E94F30563E070E039
:103BF00080E090E00E942F0C6230710581059105F4
:103C000009F080C268EC70E080E090E00E94F3056B
:103C10000E94600B8091C7039091C8031816190683
:103C20002CF401979093C8038093C7038091C70336
:103C30009091C80397FF05C001969093C8038093A5
:103C4000C7032091C7033091C803121613064CF422
:103C50008091C5039091C60301979093C60380930A
:103C6000C5038091C5039091C60397FF05C00196D7
:103C70009093C6038093C5032D32314034F08CE21B
:103C800091E09093C8038093C7038091C7039091FC
:103C9000C803843D9E4F34F484ED9EEF9093C80397
:103CA0008093C7038091C5039091C6038D329140E4
:103CB00034F08CE291E09093C6038093C503809129
:103CC000C5039091C603843D9E4F34F484ED9EEF6E
:103CD0009093C6038093C5038091C1039091C20362
:103CE0002091C5033091C603820F931F9093C203A6
:103CF0008093C1034091C3035091C4032091C70333
:103D00003091C803240F351F3093C4032093C3039D
:103D10008C30FEEF9F0734F488519A4C9093C20385
:103D20008093C1038091C1039091C203853F03E357
:103D3000900734F0885E95439093C2038093C1034B
:103D40002C301EEF310734F42851334E3093C40326
:103D50002093C3038091C3039091C403853F2AE15C
:103D6000920734F0885E9C419093C4038093C30310
:103D70000091C3031091C4031E8B0D8B24E630E029
:103D8000C801B9010E945F2D7B01E091C9030E2F8C
:103D9000EE0F110B1E830D83F801E85EF74F0091C3
:103DA000C1031091C2031C8B0B8BC801B9010E9487
:103DB0005F2D4D815E814050584F0D811E8108510D
:103DC000184F1A8709870D811E810053184F1C87D1
:103DD0000B872D813E812854384F8D819E818056DE
:103DE000984FA091BF03B091C0031A161B060CF0A8
:103DF000A6C1E4916701CE0ED11CE7FDDA94FA0169
:103E000044915B01A40EB11C47FDBA94E985FA8583
:103E100044913701640E711C47FD7A94F801449176
:103E20004B01840E911C47FD9A94F9012491E20EF6
:103E3000F11C27FDFA94FC0184918B01080F111DE0
:103E400087FD1A959301A401B701C8010E94DB0800
:103E50009601A501B301C4010E94DB089701A801E6
:103E6000B601C5010E94DB0884E00E94260A88236F
:103E700009F4A5C02091BE0328300CF0A0C0422F49
:103E8000022E000C550B8D819E81880F991FFC011D
:103E9000E05DF74FE49139E0349FD001359FB00DDC
:103EA0001124A759BC4F34E1E302F0011124159607
:103EB000FC93EE931497FC01EF5CF74FE491E3025F
:103EC000F00111241796FC93EE931697EB85FC8571
:103ED00084910B891C89080F111D87FD1A95119675
:103EE0001C930E93E985FA8584910D891E89080F2C
:103EF000111D87FD1A9513961C930E93129784E655
:103F000018968C932F5F2093BE0364E070E08CE4DE
:103F100094E00E948A0864E070E080E090E00E94F3
:103F2000F30564E070E088EE93E00E948A0864E0A4
:103F300070E080E090E00E94F30564E070E084E8C7
:103F400093E00E948A0864E070E080E090E00E94C4
:103F5000F30564E070E080E293E00E948A0864E088
:103F600070E080E090E00E94F30564E070E08CEB8C
:103F700092E00E948A0864E070E080E090E00E9495
:103F8000F30564E070E088E592E00E948A0864E04E
:103F900070E080E090E00E94F30564E070E084EF60
:103FA00091E00E948A0864E070E080E090E00E9466
:103FB000F30564E070E080E991E00E948A0800E087
:103FC00019E024E6E22EF12C802F90E0B090BE03A1
:103FD0006B2D0B2C000C770B861797070CF001C28A
:103FE000189FF001199FF00D1124E759FC4F4081F3
:103FF000518124813581420F531F51834083A28117
:10400000B381268137812A0F3B1F338322834C30B3
:10401000AEEF5A0724F448515A4C51834083189FFD
:10402000F001199FF00D1124E759FC4F4081518197
:10403000453FB3E35B0724F0485E5543518340831B
:104040002C30EEEF3E075CF4189FF001199FF00D45
:104050001124E759FC4F2851334E33832283189F94
:10406000F001199FF00D1124E759FC4F2281338193
:10407000253F4AE1340724F0285E3C413383228304
:10408000189FF001199FF00D1124E759FC4F20856E
:1040900027FF82C11086A02EAB0141505109CA2CC6
:1040A000D12CC416D5060CF064C196012F5F3F4F8A
:1040B000129FD001139FB00D1124A759BC4F2D9111
:1040C0003C9111971C9DF0011D9DF00D1124E759A5
:1040D000FC4F3183208314962D913C9115973583A5
:1040E000248312962D913C91139733832283169645
:1040F0002D913C9117973783268318962C91208712
:10410000A394CDCF1092C8031092C7031092C60398
:104110001092C50360E072E380E090E00E942F0CF3
:104120007093C2036093C10360E079E180E090E0A6
:104130000E942F0C7093C4036093C3036BCDE49172
:104140005701AE0EB11CE7FDBA94FA0144912B0160
:10415000440E511C47FD5A94E985FA854491670144
:10416000C40ED11C47FDDA94EB85FC8544911B01FC
:10417000240E311C47FD3A94F9012491E20EF11C02
:1041800027FDFA94FC018491680F711D87FD7A95D3
:10419000CE14DF0414F00C94F32BAE14BF0414F40B
:1041A0000C940B2C9E2D8F2D7601C92ED82E962F78
:1041B000872FB101292E382EAE14BF0411F5261613
:1041C000370654F0962F872F6215730514F4922D3D
:1041D000832D1B01692F782F421453042CF0641592
:1041E00075050CF4B2012101F0E4EF16F10408F0BA
:1041F0003BCE6F5F462F4419B701C2010E948A046B
:1042000033CE942D852D2B01692F782F9A2D8B2D50
:104210005701E92EF82E810104191509188F0F8B0B
:1042200086010A191B091A8F098F8B0104191509B8
:1042300018870F8387010A191B091E870D878B01B9
:1042400002191309188B0F8787010C191D091C8F80
:104250000B8FEC14FD0409F443C0860101501109D1
:104260001A8B098B8501912C812C712C612C298949
:104270003A8920173107BCF1C301698D7A8D0E94FC
:104280005F2D9B01240D351DC4016D857E850E9427
:104290005F2DCB01840D951D4F89588D640E751EC1
:1042A0006F817885860E971E821793071CF0582F12
:1042B000C901252F0034110530F441E0420F481B9D
:1042C000B8010E948A040F5F1F4FD1CF922D832D1A
:1042D0001B01692F782F9E2D8F2D76010C94182CA1
:1042E000FA8AE98ABFCFC8018C199D09AF85B889C0
:1042F0008A9F40018B9F900C9A9F900C1124C801BB
:104300008A199B09EF81F8858E9F60018F9FD00CE1
:104310009E9FD00C1124E016F1060CF4A5CDC4012B
:104320006B8D7C8D0E945F2D9B01220D331DC6017C
:104330006D857E850E945F2DCB01840D951D4F8577
:104340005889840E951E6F817885C60ED71E8217F8
:1043500093071CF0582FC901252F0034110530F4A4
:1043600041E0420F481BB8010E948A040F5F1F4FB3
:10437000D2CF169FF001179FF00D1124E759FC4F83
:104380001182108215821482138212821782168281
:104390001086BA94B092BE03189F9001199F300DF9
:1043A0001124B90167597C4F6B01DB0112968D9185
:1043B0009C91B7010E945F2D9B01F6018081918144
:1043C000B7010E945F2DCB0141E0B9010E94D208E4
:1043D000D60118968C911897845018968C930F5F7D
:1043E000F3CDD12C19E094E6692E712C4D2D50E0BF
:1043F00080916803082E000C990B481759070CF0A0
:10440000D1C1149FF001159FF00D1124E05EFC4F07
:104410002081318184819581280F391F3183208348
:104420006281738186819781860F971F9383828330
:104430002C30BEEF3B0724F428513A4C31832083C3
:10444000149FF001159FF00D1124E05EFC4F2081B8
:104450003181253F03E3300724F0285E3543318363
:1044600020838C302EEF92075CF4149FF001159F8F
:10447000F00D1124E05EFC4F8851934E93838283AC
:10448000149FF001159FF00D1124E05EFC4F828116
:104490009381853F3AE1930724F0885E9C419383A2
:1044A000828300E0149FC001159F900D1124AC0180
:1044B000405E5C4F7A015A0152E0A50EB11C202FDC
:1044C00030E06091BE03462F062E000C550BD7013D
:1044D0008D909C90F50180819181241735070CF017
:1044E00022C1129FF001139FF00D1124E759FC4FD8
:1044F00020813181281939090280F381E02DDF0103
:10450000A81BB90BCD01F901EC50FE4FE93EF34079
:1045100030F4FC01EC50FE4FE93EF34080F037FFF1
:1045200003C031952195310997FF03C0919581957D
:104530009109280F391F2C3B32400CF0F2C0202F7C
:104540004A0191E0891A9108822F90E08815990517
:10455000B4F4189FD001199FB00D1124A759BC4F76
:104560000196189FF001199FF00D1124E759FC4F97
:10457000812F01900D928A95E1F72F5FE5CF149F6F
:10458000F001159FF00D1124E759FC4F11821082A4
:10459000158214821382128217821682108661504D
:1045A0006093BE036BE470E086E990E00E948A08A5
:1045B0008091BC039091BD0302969093BD038093BC
:1045C000BC0320911F032103F0011124E157FD4F8B
:1045D000D5018D919C919183808364E670E080E0A9
:1045E00090E00E942F0C20911F032103F001112461
:1045F000E157FD4F62537109810991097583648305
:1046000064E670E080E090E00E942F0C20911F0390
:104610002103F0011124E157FD4F62537109810913
:1046200091097783668364E070E080E090E00E9407
:104630002F0C20911F032103F0011124E157FD4F9E
:1046400060872F5F20931F032103F0011124E1579E
:10465000FD4FD7018D919C9191838083D5018D91E0
:104660009C919383828364E670E080E090E00E94F6
:104670002F0C20911F032103F0011124E157FD4F5E
:1046800062537109810991097583648364E670E05E
:1046900080E090E00E942F0C20911F032103F00185
:1046A0001124E157FD4F6253710981099109778304
:1046B000668364E070E080E090E00E942F0C20911F
:1046C0001F032103F0011124E157FD4F60872F5F85
:1046D00020931F033D2D832F90E020916803422FEC
:1046E000022E000C550B4150510984179507B4F464
:1046F000189FD001199FB00D1124A05EBC4F0196E8
:10470000189FF001199FF00D1124E05EFC4F812FDE
:1047100001900D928A95E1F73F5FDDCF2150209304
:1047200068030F5FCCCEB3010E945F2DFB01C40173
:10473000B3010E945F2DCB01D70118962C91213037
:1047400009F144F4222391F025E045E0BF010E94E5
:104750003C0A16C02230F1F02330B1F7BF01685097
:10476000710900E120E140E257E007C0BF01685055
:10477000710900E120E140E857E008970E94C10478
:10478000D39434CEBF016850710900E120E140E6C6
:1047900057E0F3CFBF016850710900E120E140E428
:1047A00057E0EBCFD12C19E084E6682E712C4D2D0B
:1047B00050E080911F03082E000C990B48175907F1
:1047C0000CF0D6C1149FF001159FF00D1124E15794
:1047D000FD4F2081318184819581280F391F3183DC
:1047E00020836281738186819781860F971F9383CF
:1047F00082832C30BEEF3B0724F428513A4C31839E
:104800002083149FF001159FF00D1124E157FD4FF7
:1048100020813181253F03E3300724F0285E3543B2
:10482000318320838C302EEF92075CF4149FF001CB
:10483000159FF00D1124E157FD4F8851934E93833E
:104840008283149FF001159FF00D1124E157FD4F55
:1048500082819381853F3AE1930724F0885E9C41F1
:104860009383828300E0149FC001159F900D112453
:10487000AC0141575D4F7A015A0152E0A50EB11CBF
:10488000202F30E06091BE03462F062E000C550B02
:10489000D7018D909C90F501808191812417350777
:1048A0000CF027C1129FF001139FF00D1124E7595E
:1048B000FC4F20813181281939090280F381E02DD4
:1048C000DF01A81BB90BCD01F901E057FE4FE13222
:1048D000F34030F4FC01E057FE4FE132F34080F04A
:1048E00037FF03C031952195310997FF03C091959A
:1048F00081959109280F391F283532400CF0F7C0F7
:10490000202F4A0191E0891A9108822F90E08815A2
:104910009905B4F4189FD001199FB00D1124A7591F
:10492000BC4F0196189FF001199FF00D1124E75913
:10493000FC4F812F01900D928A95E1F72F5FE5CF13
:10494000149FF001159FF00D1124E759FC4F1182BF
:1049500010821582148213821282178216821086A8
:1049600061506093BE036BE470E086E990E00E94C2
:104970008A088091BC039091BD0304969093BD0377
:104980008093BC0320918E022103F0011124E2598F
:10499000FE4FD7018D919C9191838083D5018D919C
:1049A0009C919383828364E670E080E090E00E94B3
:1049B0002F0C20918E022103F0011124E259FE4FA9
:1049C00062537109810991097583648364E670E01B
:1049D00080E090E00E942F0C20918E022103F001D4
:1049E0001124E259FE4F62537109810991097783BD
:1049F000668364E070E080E090E00E942F0C2091DC
:104A00008E022103F0011124E259FE4F60872F5FCF
:104A100020938E022103F0011124E259FE4FD701A9
:104A20008D919C9191838083D5018D919C919383ED
:104A3000828364E670E080E090E00E942F0C209179
:104A40008E022103F0011124E259FE4F62537109D5
:104A5000810991097583648364E670E080E090E0E9
:104A60000E942F0C20918E022103F0011124E259A3
:104A7000FE4F62537109810991097783668364E06F
:104A800070E080E090E00E942F0C20918E022103C4
:104A9000F0011124E259FE4F60872F5F20938E02B0
:104AA0003D2D832F90E020911F03422F022E000CFA
:104AB000550B4150510984179507B4F4189FD00144
:104AC000199FB00D1124A157BD4F0196189FF001F9
:104AD000199FF00D1124E157FD4F812F01900D9288
:104AE0008A95E1F73F5FDDCF215020931F030F5FD1
:104AF000C7CEB3010E945F2DFB01C401B3010E9428
:104B00005F2DCB01D70118962C91213009F144F487
:104B1000222391F024E044E0BF010E943C0A16C029
:104B20002230F1F02330B1F7BF016450710908E081
:104B300028E040E057E007C0BF016450710908E079
:104B400028E048E157E004970E94C104D3942FCE97
:104B5000BF016450710908E028E040E157E0F3CF5D
:104B6000BF016450710908E028E048E057E0EBCF4E
:104B7000D12C19E004E6A02EB12C4D2D50E08091EF
:104B80008E02082E000C990B481759070CF026C10D
:104B9000149FF001159FF00D1124E259FE4F208162
:104BA000318184819581280F391F3183208362816F
:104BB000738186819781860F971F938382832C3020
:104BC000BEEF3B0724F428513A4C31832083149FD5
:104BD000F001159FF00D1124E259FE4F2081318123
:104BE000253F03E3300724F0285E354331832083DB
:104BF0008C302EEF92075CF4149FF001159FF00D9E
:104C00001124E259FE4F8851934E93838283149F5F
:104C1000F001159FF00D1124E259FE4F828193811E
:104C2000853F3AE1930724F0885E9C419383828319
:104C300000E0149FC001159F900D1124AC01425952
:104C40005E4F7A014A0152E0850E911C202F30E020
:104C50006091BE03462F062E000C550BD701ED9137
:104C6000FC91D4018D919C91241735070CF078C0EC
:104C7000129FD001139FB00D1124A759BC4F2D9145
:104C80003C9111972E1B3F0B28533F4F2139314048
:104C900008F064C012962D913C91D901A81BB90B64
:104CA000CD0188539F4F8139914008F057C0202F84
:104CB00041505109822F90E084179507B4F4189F52
:104CC000D001199FB00D1124A759BC4F0196189F10
:104CD000F001199FF00D1124E759FC4F812F01902D
:104CE0000D928A95E1F72F5FE5CF61506093BE0387
:104CF0006BE470E086E990E00E948A088091BC0332
:104D00009091BD0308969093BD038093BC033D2D05
:104D1000832F90E020918E02422F022E000C550B23
:104D20004150510984179507B4F4189FD001199F79
:104D3000B00D1124A259BE4F0196189FF001199F82
:104D4000F00D1124E259FE4F812F01900D928A95AA
:104D5000E1F73F5FDDCF215020938E020F5F76CFCA
:104D6000B5010E945F2D4B01CF01B5010E945F2D5F
:104D7000CB01F7012085213009F144F4222391F081
:104D800022E042E0B4010E943C0A16C02230F1F059
:104D90002330B1F7B4016250710904E024E040EE21
:104DA00056E007C0B4016250710904E024E048EF06
:104DB00056E002970E94C104D394DFCEB401625042
:104DC000710904E024E040EF56E0F3CFB4016250F3
:104DD000710904E024E048EE56E0EBCF0E94490C54
:104DE000E0916D018091B2039091B303EE2309F439
:104DF00015C2E150E0936D012091CB033091CC03BB
:104E00004091CD035091CE03B901615273406F3B85
:104E10007B4258F4BA01615971406F3D754128F4E5
:104E2000E11103C061E060936D016091CF03709167
:104E3000D003260F371F3093CC032093CB03609110
:104E4000D1037091D203460F571F5093CE03409366
:104E5000CD03293C12E3310734F0285E354330930B
:104E6000CC032093CB032091CB033091CC032C3087
:104E70006EEF360734F428513A4C3093CC0320932C
:104E8000CB03453F7AE1570734F0485E5C415093CD
:104E9000CE034093CD032091CD033091CE032C302F
:104EA000AEEF3A0734F42851334E3093CE032093BB
:104EB000CD0320916C011216FCF4409164015091D5
:104EC00065016091680170916901460F571F509309
:104ED00065014093640140916601509167016091C2
:104EE0006A0170916B01460F571F50936701409301
:104EF0006601245020936C016EE170E00E944B2DFE
:104F0000892B21F564E670E080E090E00E942F0C90
:104F100062537109810991097093D0036093CF03A3
:104F200064E670E080E090E00E942F0C625371090B
:104F3000810991097093D2036093D10368E170E015
:104F400080E090E00E942F0C6093D3038091B20325
:104F50009091B30369E670E00E944B2D892B79F59F
:104F60008091CB039091CC03909365018093640171
:104F70008091CD039091CE03909367018093660159
:104F8000E091D3032E2F220F330BF901E05DF74F91
:104F9000849144E18402C0011124909369018093BB
:104FA0006801F901EF5CF74FE491E402F00111248C
:104FB000F0936B01E0936A0184E680936C01109199
:104FC0006C0111160CF471C010926C0110926B01FF
:104FD00010926A01109269011092680110926701A3
:104FE00010926601109265011092640110E009E0D0
:104FF000812F90E04091BE03642F042E000C770BAC
:105000002091CB033091CC03861797070CF0A1C0F9
:10501000089FF001099FF00D1124E759FC4F808192
:105020009181821B930B22813381E091CD03F0911A
:10503000CE032E1B3F0BFC01EC50FE4FE93EF3402C
:1050400030F4F901EC50FE4FE93EF34080F097FF59
:1050500003C091958195910937FF03C03195219542
:105060003109820F931F8C3B92400CF070C0212FAE
:1050700061507109822F90E08617970784F5089F89
:10508000D001099FB00D1124A759BC4F0196089F6C
:10509000F001099FF00D1124E759FC4F802F01907A
:1050A0000D928A95E1F72F5FE5CF8091660190918F
:1050B0006701E4E6F0E0BF010E945F2D9B01809153
:1050C000640190916501BF010E945F2DCB0141E019
:1050D000B9010E94D208145010936C0187CF41503F
:1050E0004093BE036BE470E086E990E00E948A087A
:1050F0008091BC039091BD0305969093BD0380936E
:10510000BC0310926C0110926B0110926A01109214
:105110006901109268011092670110926601109265
:105120006501109264011092D3031092D203109281
:10513000D1031092D0031092CF031092CE0310929D
:10514000CD031092CC031092CB0310926D011F5F20
:105150004FCF12161306C4F48091CD039091CE0365
:1051600004E610E0B8010E945F2DFB013497C901ED
:10517000B8010E945F2DCB0108E028E045EA58E025
:10518000BF0104970E94C10481E080930D0182E079
:1051900090E09093B7038093B6030AE010E0109379
:1051A000B5030093B4036091BC037091BD0390E01C
:1051B00080E04AE00E94840B80E290E09093B70385
:1051C0008093B6031093B5030093B4038091BB039F
:1051D000082E000C990B0E94D20B88E790E0909368
:1051E000B7038093B6031093B5030093B403809183
:1051F000CA03082E000C990B0E94D20B8091CA039F
:10520000811102C00E94360B88E00E94260A882382
:1052100011F40C94821B84E00C94871D6EE170E005
:105220000E944B2D892B09F0AFCF8091BF03909145
:10523000C0038837910509F0A7CF6AE070E080E0ED
:1052400090E00E942F0C683071058105910509F0EE
:105250009BCF80EF80936D0168EE7CE180E090E071
:105260000E942F0C60587A4D7093CC036093CB034F
:1052700068E670E180E090E00E942F0C60547D4E63
:105280007093CE036093CD0364E670E080E090E01D
:105290000E942F0C62537109810991097093D00308
:1052A0006093CF0364E670E080E090E00E942F0CF2
:1052B00062537109810991097093D2036093D103FC
:1052C00063CF68EB7BE080E090E00E94F3050E94F2
:1052D000360B82E00C94871DB4E6EB2EF12C00E037
:1052E000BE016D5F7F4FC7010E941B0C8B819C81AB
:1052F000019611F41C821B82D02E2091BC033091A8
:10530000BD038B819C818217930708F099C180E2CD
:105310008093B8038093B9038093BA0310E051E2FD
:10532000C52E60E3B62E71E4A72EEFE29E2EFAE5BD
:105330008F2EAFE37A2E13300CF01AC10E940D0BA2
:105340008823C9F3E0E1F0E0F093B703E093B603FC
:105350001092B5031092B40385ED96E00E940B0AFB
:1053600028E530E03093B7032093B6031092B503DD
:105370001092B4036091BC037091BD0390E080E093
:105380004AE00E94840B48E350E05093B7034093F7
:10539000B60364E170E07093B5036093B403809149
:1053A000B8030E94060A80E490E09093B7038093CC
:1053B000B603A4E1B0E0B093B503A093B403809129
:1053C000B9030E94060AE8E4F0E0F093B703E09323
:1053D000B60324E130E03093B5032093B403809109
:1053E000BA030E94060A2BE130E04EE350E06BE185
:1053F00070E088E390E00E94DB082BE130E046E4B7
:1054000050E06BE170E080E490E00E94DB082BE16B
:1054100030E04EE450E06BE170E088E490E00E9400
:10542000DB08812F012E000C990B079643E0880FB3
:10543000991F4A95E1F7AC014A5F5F4F2CE130E0DC
:105440006CE170E00E94DB0866E970E080E090E0CB
:105450000E94F30580E20E94260A882349F068EC46
:1054600070E086E194E00E948A08115008F410E090
:1054700080E40E94260A882351F01F5F133009F44C
:1054800012E068EC70E086E194E00E948A0880E116
:105490000E94310A882339F1812F012E000C990BCB
:1054A000AC0148545C4F7A01DA018C918F5F8C9388
:1054B00066E970E08BE092E00E948A08F701808143
:1054C000803311F480E28083D7018C91813209F41A
:1054D000AC92F70180818B3509F4B082D7018C91B1
:1054E000803409F4CC9280E80E94310A882331F19B
:1054F000812F012E000C990BFC01E854FC4F7F0119
:1055000080818150808366E970E08BE092E00E94A8
:105510008A08D7018C91803209F47C92F70180814E
:105520008F3209F48082D7018C918F3109F49C92DB
:10553000F7018081803411F480E2808388E00E944A
:10554000310A882349F0123039F468EC70E086E1C2
:1055500094E00E948A0813E08091630180936201C5
:105560000E94A9088093630181E00E946905E3CE4F
:10557000F5E00F9F800111240A591F4F580122E0C6
:10558000A21AB108BE016D5F7F4FC5010E941B0CBE
:105590008B819C81019611F41C821B82C8010E94A0
:1055A000190C682E48014FEF841A940AC4010E9416
:1055B000190C782E780152E0E50EF11CC7010E940B
:1055C000190CC82EBA82A9826091BC03CE01019643
:1055D0000E94000CC80101979A8389836091BD03E2
:1055E000CE0101960E94000C6091B803C8010E9490
:1055F000DA2C6091B903C4010E94DA2C6091BA03DD
:10560000C7010E94DA2C8B819C819093BD0380930B
:10561000BC036092B8037092B903C092BA03D394EA
:105620000B5F1F4F67E0D612A9CF80E28093B803CB
:105630008093B9038093BA030E944D0B0C94821B94
:1056400075E0E70EF11C0F5F073009F049CEF4CF8B
:1056500080E290E09093B7038093B6031092B50375
:105660001092B40381E080930D014BE050E067E3BA
:1056700071E08DE498E00E949D0629E0C22ED12CB5
:1056800004E610E0F12CE12C3EE1A32EB12C6CEBF2
:1056900073E0C8010E941B0C8091BC039091BD0374
:1056A000019621F41092BD031092BC03C80102962A
:1056B0000E94190C8093B803C80103960E94190C2C
:1056C0008093B903C80104960E94190C8093BA0311
:1056D000B092B703A092B603D092B503C092B403C0
:1056E000BFEFEB1AFB0AC7010E94D20B83EA98E0D6
:1056F0000E940B0A8091B8030E94060A8091B903A8
:105700000E94060A8091BA030E94060A81EA98E084
:105710000E940B0A6091BC037091BD0390E080E091
:105720004AE00E94840B1092BD031092BC030B5FF1
:105730001F4FE8E0CE0ED11CF7E0EF16F10409F0A0
:10574000A6CF88E00E94260A81111092D40380E23D
:105750000E94260A882311F40C94821B85E00C9485
:10576000871D80E290E09093B7038093B6038EE1AB
:1057700090E09093B5038093B40382E080930D0191
:105780008BE998E00E940B0A84E00E94260A882395
:1057900019F081E08093D40388E00E94260A8111E9
:1057A0000E944D0B80E80E94260A811107C080E10B
:1057B0000E94260A882311F40C94821B8091B10365
:1057C000882371F00E94B1086091B10382E090E0FB
:1057D0009A838983CE0101960E94000C0C94821B4F
:1057E0000E94B608F1CFAC14BD0414F00C94DC2078
:1057F000AE14BF0414F40C946621942D852D210160
:105800001B01692F782F9C2D8D2D67017501A92E05
:10581000B82E0C94D220AC14BD0414F40C940B21BB
:10582000942D852D2101292E382E9A2D8B2D560150
:10583000C92ED82E0C940B218F929F92AF92BF92BB
:10584000CF92DF92EF92FF92CF93DF93EC016881CA
:1058500079818A819B81611571058105910521F40A
:1058600064E279ED8BE597E02DE133EF41E050E024
:105870000E94E82C49015A019B01AC01A7EAB1E45E
:105880000E94072D6B017C01ACEEB4EFA5019401E1
:105890000E94152DC60ED71EE81EF91EF7FE06C083
:1058A00081E0C81AD108E10880E8F80AC882D982E4
:1058B000EA82FB82C701B6019F77DF91CF91FF900B
:1058C000EF90DF90CF90BF90AF909F908F90089512
:1058D0008F929F92AF92BF92CF92DF92EF92FF9200
:1058E00060910E0170910F01809110019091110152
:1058F000611571058105910521F464E279ED8BE56F
:1059000097E02DE133EF41E050E00E94E82C49019F
:105910005A019B01AC01A7EAB1E40E94072D6B017B
:105920007C01ACEEB4EFA50194010E94152DC60ECA
:10593000D71EE81EF91EF7FE06C081E0C81AD1087E
:10594000E10880E8F80AC0920E01D0920F01E092BF
:105950001001F0921101C701B6019F77FF90EF90FF
:10596000DF90CF90BF90AF909F908F9008956093FD
:105970000E0170930F01809310019093110108950F
:10598000F999FECF92BD81BDF89A992780B5089507
:10599000262FF999FECF92BD81BDF89A019700B4E8
:1059A000021639F01FBA20BD0FB6F894FA9AF99A88
:1059B0000FBE0895262FF999FECF1FBA92BD81BD63
:1059C00020BD0FB6F894FA9AF99A0FBE0196089581
:1059D000052E97FB1EF400940E94FF2C57FD07D064
:1059E0000E941A2D07FC03D04EF40C94FF2C509506
:1059F0004095309521953F4F4F4F5F4F08959095BB
:105A00008095709561957F4F8F4F9F4F08950E94AD
:105A10003C2DA59F900DB49F900DA49F800D911DCE
:105A200011240895B7FF0C94072D0E94072D821BA7
:105A3000930B0895A1E21A2EAA1BBB1BFD010DC0FA
:105A4000AA1FBB1FEE1FFF1FA217B307E407F5072E
:105A500020F0A21BB30BE40BF50B661F771F881F0A
:105A6000991F1A9469F760957095809590959B01A0
:105A7000AC01BD01CF010895A29FB001B39FC00149
:105A8000A39F700D811D1124911DB29F700D811D6A
:105A90001124911D0895AA1BBB1B51E107C0AA1F29
:105AA000BB1FA617B70710F0A61BB70B881F991FBF
:105AB0005A95A9F780959095BC01CD01089597FB63
:105AC000072E16F4009407D077FD09D00E944B2DC5
:105AD00007FC05D03EF4909581959F4F08957095F1
:105AE00061957F4F0895EE0FFF1F0590F491E02D13
:065AF0000994F894FFCFB9
:105AF600FFFFFFFF00E100000000000010010100B1
:105B0600000000C18081000000000000004D07CAAF
:105B1600066E076307B40772079007000000005F70
:105B2600099D06810B800B484947482053434F5235
:045B360045530000D3
:00000001FF
